:020000040000FA
:02000000B7291E
:02000800B42D15
:10001000831203134C08E1000130E2004D0803197C
:100020001528E20D6210FF3E0F286208E300E20986
:1000300080304C07840062088005841362088005C4
:100040000800C920E830F4000330F500F601F7019C
:10005000D2204E08F4004F08F500F601F701FE200B
:10006000F30CF20CF10CF00CF313F30CF20CF10C9A
:10007000F00CF313F30CF20CF10CF00CF31370080A
:10008000E4007108E500C9205008F4005108F500AB
:10009000F601F701D2206408F4006508F500F601C6
:1000A000F7010330003E03195C28F40DF50DF60D41
:1000B000F70D7410FF3E5328FE207008E800710809
:1000C000E9007208EA007308EB000A30F40000301F
:1000D000F5006408F0006508F10087217008E4006D
:1000E0007108E50000307102031D782803307002AA
:1000F00003187B280800610884006B08003C031D7E
:100100008B286A08003C031D8B286908003C031DEE
:100110008B286808003C0318C6286308800465081B
:100120000319A228E601E70166086702031D9A2861
:10013000650866020318A228EC01A421E60A031947
:10014000E70A94286408EC00A42162088005650889
:100150000319BA28E601E70166086702031DB22801
:10016000650866020318BA28EC01A421E60A0319FF
:10017000E70AAC286408EC00A4210130E802031C63
:10018000E902031CEA02031CEB027D2862088005D9
:100190000800831203130030F0003230F100F20146
:1001A000F3010800831203132230FC00F801F90167
:1001B000FA01FB01FC030319EE280310FB0CFA0CF7
:1001C000F90CF80CF30CF20CF10CF00C031CDA280F
:1001D000FC030319ED28EF20DE28EF200800740847
:1001E000F80775080318750FF90776080318760FD6
:1001F000FA0777080318770FFB0708008312031329
:10020000FB01FA01F901F801E001730DF80D740822
:100210006321F30D0730FC00730D5D217408731C1E
:100220001329632114297521F30DFC0B0C29720D80
:100230005D217408731C1E2963211F297521F20D8D
:100240000730FC00720D5D217408721C292963219E
:100250002A297521F20DFC0B2229710D5D217408EC
:10026000721C3429632135297521F10D0730FC00FA
:10027000710D5D217408711C3F296321402975218E
:10028000F10DFC0B3829700D5D217408711C4A2991
:1002900063214B297521F00D0730FC00700D5D21A5
:1002A0007408701C5529632156297521F00DFC0B2B
:1002B0004E2970185C29EF200800F80DF90DFA0D91
:1002C000FB0DE00D0800F8027508031C750FF9021C
:1002D0007608031C760FFA027708031C770FFB02DF
:1002E0000301031C0130E0020800F8077508031839
:1002F000750FF90776080318760FFA0777080318C1
:10030000770FFB07030103180130E0070800831291
:100310000313F801F9011030FC00710DF80DF90D0F
:100320007408F8027508031C750FF90203189F2959
:100330007408F80775080318750FF9070310F00D16
:10034000F10DFC0B8D29080083120313EC03EC0361
:100350006C08003C0318B129EC0300000000000009
:10036000A82900000000000000000000080083121F
:1003700085018601870183160C10D13081000B3076
:100380008500051500308600F030870005309F009D
:10039000831220308B0080309F000530CC0002306B
:1003A000CD000820D201203084000530C40003179E
:1003B00026308D00031783160C1483120C088D0A47
:1003C00003138000840AC40BDA29A501B601B70122
:1003D000A801A901AA01BB018B17FF3086002A22C0
:1003E0004B225622BC30B0000230B1004030B20087
:1003F000DD30A7002810A5013030BD0050240330A7
:100400002502031CFC29FF308600A50101302502CE
:10041000031C062AB001B101B201FC30A70028106C
:100420003030BD000630A9001A30AA00502499309F
:1004300030020319202A1130B007B107B207102A81
:10044000FF308600A50101302502031C232AA501E7
:10045000B801A82A1030CE000330CF006430D0009D
:100460000030D10083160511831221208316051553
:1004700083121E30A3251730CE000430CF00643025
:10048000D0000030D100831605118312212083167D
:100490000515831208000030502210305022203001
:1004A00085006B228C227B229B2208000330C50032
:1004B00085016B228C22103085008C222030850033
:1004C0008C227B229B22103085009B2285019B225F
:1004D000C50B582A08008701FE30C1000830C4004F
:1004E000FF308600410886000A30A3250314C10DA1
:1004F000C40B702A08000F3087007F30C10008301D
:10050000C400FF308600410886000A30A32503148A
:10051000C10CC40B812A0800C0011030C400FF3098
:100520008600400887007F3086000A30A325C00A75
:10053000C40B8F2A08001030C400FF30860044032B
:100540008700FE3086000A30A325C40B9D2A0800D0
:10055000A8194F236D23003036020319B32A043043
:100560003602031DBF2A9D23FE30A700391CF92A3D
:100570003D0884000008F0390319A713F92A013057
:100580003602031DC82A2030BD00FD30A700F92A1D
:1005900002303602031DD82A83233030BD003D309F
:1005A000A70010303102031CA7120A30B204F92A46
:1005B000FB302507031CB32AF6302507031CC32A8A
:1005C000E0302507031CB32ADB302507031CCC2AA7
:1005D000CB302507031CB32AC6302507031CC32ACA
:1005E000B0302507031CB32AAB302507031CCC2AE7
:1005F000B32A5024521C0C2B7030CE000330CF0095
:100600006430D0000030D100831605118312212000
:100610008316051583121D2BD21C1D2BE030CE0036
:100620000630CF00E830D0000330D100831605112A
:1006300083122120831605158312D201BB1F272B9D
:10064000B60A053036020319B601B7173E2B3B1F19
:100650002B2BC6233E2B3B1E3E2B06302402031CB5
:10066000382B55302402031C3E2B8B13F925392BD4
:100670008B13A401A501A901AA018B17BB01A81C1A
:10068000A82AFD24A810A81501302202031DA82ABB
:100690003F2501302102031DA82A5125A82AA811AF
:1006A000203084000530C400031726308D0003136A
:1006B0000008840A03178C0083168C130C15553020
:1006C0008D00AA308D008C148C18642B0C118312B1
:1006D0008D0A0313C40B582B080083169F13831233
:1006E00081309F009A251F151F19742B76301E022A
:1006F00003187C2B2815812B8A301E02031C812BAA
:1007000028111F10080083169F17831289309F003D
:100710009A251F151F198A2B1E08AB0083161E0869
:100720008312AC001F1024263208B100B10E33082A
:10073000B1043408B200B20E0800B90183160515E1
:10074000831223300519C42B2308B0002408B100FC
:100750002508B20039143008031DB12B1230B00047
:10076000C32B12303002031CC32BB9140319C32B43
:10077000B0000E303002031CC32B103030020318BF
:10078000C32B0630B0023030BD0008008B1305309B
:10079000B600B7132008AD002108AE002208AF0054
:1007A0002030BD00C130A7005024BB1B1F2C3B1BB9
:1007B000E12BBB1EDD2B5125D22B3B1ED22B7E25E0
:1007C000D22B3130A7005024BB1BD22B3B1BF22B6A
:1007D000BB1EEC2B3F25E12B3B1EE12B7225E12BB1
:1007E0002030BD000D30A7005024BB1BE12B3B1B6C
:1007F000012CBB1EFD2BFD24F22B3B1EF22B622590
:10080000F22B9D23C230A7005024BB1BF02B3B1BB7
:100810001F2CBB1E132C23308400032624302302FC
:100820000318A301012C3B1E012C233084008F25CB
:10083000F9302302031D012C2330A300012C9D233A
:100840003230A7005024BB1B012C3B1B3D2CBB1E90
:10085000312C243084000326603024020318A401C4
:100860001F2C3B1E1F2C243084008F25F9302402BE
:10087000031D1F2C5930A4001F2C20082D02031D1E
:10088000492C21082E02031D492C22082F0203198E
:100890004A2CA815B601A901AA01A5018B170800C9
:1008A00005303602031D552CBB0185013D0884002F
:1008B000B71B5C2CA71F612CC001B71BC017000E13
:1008C000C324271F672C0830C0000008C324103041
:1008D0008500840AA71E6F2CC001000EC324271EAA
:1008E000752C0830C0000008C32420308500840A1D
:1008F000A71D7D2CC001000EC324271D832C0830AA
:10090000C0000008C324FF30860030308500A71CDB
:100910009D2C0F30391CA82C05303602031D952C58
:100920000B30B91CA82C0730A82C0F303A1CA82C6F
:100930000730B91CA82C0B30A82C0030271CA82C81
:10094000053036020319A72C0130271FA82C0530CB
:10095000FF3A86009C25FF308600BC080319B22CA4
:10096000BC03BB2C0708F039F03ABB000319BB2CC1
:100970009630BC002814053036020319C22C281CFE
:10098000502C281008000F39C300C01BD22C063091
:10099000C2000310C30DC30DC30D5630C3070318A7
:1009A000C20ADD2C3608C400C40AFE30C600C403E7
:1009B0000319DD2C0314C60DD72C0830C400FF30FA
:1009C0008600281DE42C9E2540087F398700C01B27
:1009D000ED2CF924C60004308A00460886009C25C8
:1009E000C00AC30A0319C20AC40BDF2CFF308600F9
:1009F000080042088A0043088200A20A2208A600D2
:100A00000F30A6050A302602031D082D0630A20766
:100A10001225A60022082602031C0F2D0800013013
:100A2000A200080002302102031D2B2D200E0F39D9
:100A3000A6000310A60DA60DA607A60D20080F39C7
:100A400026070339031D272D2008031D292D2830D3
:100A50003E2D29303E2D0430210203193D2D063054
:100A6000210203193D2D0930210203193D2D1130BA
:100A7000210203193D2D31303E2D30300800A10AEE
:100A80002108A6000F30A6050A302602031D4A2DB4
:100A90000630A10713302102031C502D0130A100A4
:100AA0000800A00A2008A6000F30A6050A3026027A
:100AB000031D5C2D0630A007A0302002031C612D11
:100AC000A0010800A20303196F2D2208A6000F3011
:100AD000A6052602031D08000630A2020800122502
:100AE000A2000800A103031D772D12307C2D0F30CA
:100AF0002102031D08000930A1000800A003FF30F7
:100B00002002031D852D66308D2D2008A6000F3094
:100B1000A6052602031D08000630A0020800800377
:100B20000008B5000F30B5053502031D080006307A
:100B30008002080016309F2D34309F2D6930BE0092
:100B4000BE0BA02D0800BE000030BF00000000005A
:100B50000000000000000000000000000000BF0BCB
:100B6000A62DBE0BA42D0800FD00030E8301FE0080
:100B70000A08FF008A010408ED000B19C02DE02DC2
:100B80000B11AA0FC42DA90A232635302A02031DF2
:100B9000E02D0C302902031CE02D0130BA06A9011A
:100BA000AA01E925281438080319DA2DB80BDE2D1F
:100BB000B713DE2DB71FDE2D0230B8000F26E02D53
:100BC0006D0884007F088A007E0E8300FD0E7D0E76
:100BD000090025308400032660302502031C08002C
:100BE000A50124308400032660302402031C080081
:100BF000A40123308400032624302302031C0800B0
:100C0000A814A3010800800A0008B5000F30B5053C
:100C10000A303502031D0800063080070800043042
:100C20003602031D222E59302402031D1D2E57307B
:100C30002502031C1D2E5214222E25082404031DF8
:100C4000222ED214080008002B0E0F39F03EB100FE
:100C5000B107E23EB200323EB4002B080F39B207B2
:100C6000B207B407E93EB300B307B3072C0E0F3940
:100C7000B307B407B30DB40DB409B40D2C080F3984
:100C8000B407B10D0730B0000A30B407B303031C3A
:100C9000452EB307B203031C492EB207B103031C50
:100CA0004D2EB107B003031C512E080081340034CF
:100CB0007E347E347E3400348134FF34FF34FF349C
:100CC000BE3400340034FE34FF34FF349E341C3410
:100CD0007834723466340E349E34FF34B934383488
:100CE0006E346E3446341034B934FF34E334C334D4
:100CF000BB3400340034FB34FB34FF340D340C348B
:100D00006E346E346E346034F134FF348134003428
:100D10006E346E346E342034B134FF343F343F349B
:100D20007834703467340F341F34FF349134103406
:100D30006E346E346E3410349134FF348D34043498
:100D400076347634763400348134FF343F343F34A3
:100D5000C1348034BE34BE34BE34DD340734033491
:100D6000F934FC34F93403340734FF34F134EA3411
:0C0D7000EA34F334FF34E034F734EF349D
:02400E00723FFF
:1042000043006F0070007900720069006700680069
:1042100074002000280043002900200032003000F4
:10422000300037002D00320030003100390020000E
:104230006200790020004D002E00590061006D00E1
:1042400061006D006F0074006F00FF001400090032
:0642500001000000000067
:00000001FF
